:03000000023CD3EC
:0C3CD30078FFE4F6D8FD75816A023D1A06
:10169A0020000A3C2E2E2E3E004950436F6E6E6586
:1016AA0063745245510A004950436F6E6E65637404
:1016BA00000A49504E6F41434B210A003E432C56C3
:1016CA002C43432CC0E4E0EFF2E5F020D1E8EDEA48
:1016DA00EEEC49500A003E432C4D41432C25303252
:1016EA0062583A25303262583A25303262583A25E1
:1016FA00303262583A25303262583A2530326258CE
:10170A002C4D414320E0E4F0E5F10A003E432C561B
:10171A0045522C20332E3220EEF2202573202573D9
:10172A002CC2E5F0F1E8FF20495020ECEEE4F3EB9F
:10173A00FF0A004A616E20323620323031320031DF
:10174A00333A30333A3035003E432C4C442C505215
:10175A004F473A202020202020202020202020200F
:10176A00202020202020202020202020202020206F
:10177A00202020202020202020202020202020205F
:10178A00202020202020202020202020202020204F
:10179A0020202020202020202CC4E0F2E020EFF09E
:1017AA00EEF8E8E2EAE828F4E0E9EB290A003E2A42
:1017BA002C312CCEF1EDEEE2EDFBE520EFE0F0E08E
:1017CA00ECE5F2F0FB20F1E5F2E5E2EEE3EE20E8EB
:1017DA00EDF2E5F0F4E5E9F1E00A003E412C413092
:1017EA00312C2562752E2562752E2562752E25628D
:1017FA00752C495020E0E4F0E5F120E0E4E0EFF256
:10180A00E5F0E00A003E412C4130322C2562752E6B
:10181A002562752E2562752E2562752C495020E0A9
:10182A00E4F0E5F120EEF1ED2E20F1E5F0E2E5F04D
:10183A00E00A003E412C4130332C2562752E256288
:10184A00752E2562752E2562752C495020E0E4F02C
:10185A00E5F120F0E5E72E20F1E5F0E2E5F0E00A17
:10186A00003E412C4130342C2562752E2562752E9E
:10187A002562752E2562752CCCE0F1EAE020F1E5AF
:10188A00F2E80A003E412C4130352C2562752E259E
:10189A0062752E2562752E2562752CD8EBFEE70A35
:1018AA00003E2A2C312CC4EEEF2E20EFE0F0E0ECC3
:1018BA00E5F2F0FB20F1E5F2E5E2EEE3EE20E8EDF9
:1018CA00F2E5F0F4E5E9F1E00A003E422C5330314A
:1018DA002C2562752CC6E4E0F2FC20E7E0EFF0EE7E
:1018EA00F1E020F1EEE5E4E8EDE5EDE8FF20EEF2C7
:1018FA0020F1E5F0E2E5F0E00A003E422C533032F6
:10190A002C2562752CCEE1ECE5ED20F120F1E5F015
:10191A00E2E5F0EEEC20E1E5E720EAE2E8F2E0EDCC
:10192A00F6E8E90A003E422C5330332C2562752C26
:10193A00CFE5F0E5E7E0EFF3F1EA20EFF0E820EF9A
:10194A00EEF2E5F0E520F1E2FFE7E820F120F1E52B
:10195A00F0E2E5F0EEEC0A003E422C5330382C253A
:10196A0062752CCCE5E4EBE5EDEDFBE9204950206E
:10197A00EAE0EDE0EB28E7E0E4E5F0E6EAE020E47F
:10198A00EE203520F1E5EA290A003E422C53303593
:10199A002C2562752CCAE0EDE0EB20F8E8F0EEEABF
:1019AA00EEE2E5F8E0F2E5EBFCEDEEE3EE20EEE147
:1019BA00ECE5EDE00A003E532C5330362C2530324C
:1019CA0062582530326258253032625825303262E8
:1019DA0058253032625825303262582C4D41432006
:1019EA00E0E4F0E5F120F8E8F0EEEAEEE2E5F8E00E
:1019FA00F2E5EBFCEDEEE3EE20EEE1ECE5EDE00ADC
:101A0A00003E454E440A000A44756D705820202055
:101A1A002020303020303120303220303320303412
:101A2A0020303520303620303720303820303920E9
:101A3A00304120304220304320304420304520308D
:101A4A0046000A3A003A20000A000A44756D7044BA
:101A5A0020202020203030203031203032203033F6
:101A6A0020303420303520303620303720303820AE
:101A7A003039203041203042203043203044203059
:101A8A004520304600457272206B65790052642009
:101A9A00656570726F6D0A005264204D454D0A00EB
:101AAA00526420436F64650A005772697465204363
:101ABA006F64650A0044656275674950204F4E0A93
:101ACA000044656275674950204F46460A004465DE
:101ADA0062756755736572204F6E0A0044656275B8
:101AEA006755736572204F46460A004465627567FA
:101AFA004D7367204F6E0A0044656275674D7367C0
:101B0A00204F46460A00436F6E666967206C6F6312
:101B1A006B210A00577220656570726F6D0A00208A
:101B2A005361766520656570726F6D210A00457292
:101B3A0072204D414321004C6F61643E3E002A00F1
:101B4A00CEF8E8E1EAE00A00202D2025752825755F
:101B5A00290A003C4130313D003C4130323D003CD5
:101B6A004130333D003C4130343D003C4130353D4D
:101B7A00003C21003C5330313D003C5330323D00A3
:101B8A003C5330333D003C5330353D003C533038F4
:081B9A003D003C5330363D00D4
:063A2100016700016500D1
:10464400C28E438910E4F58B758DB8D2ABD28E221D
:03001B00023C4361
:103C4300C0E0C083C082C0D0C28E758B00758DB8B2
:103C5300201C0675A61E75A6E10565D218E56760EA
:103C6300020567056AE56A540F7051E566D394014E
:103C730040021566D224E56A543F7012D21690664C
:103C83008EE0600A04F0E0D394B44002D21C906644
:103C930087E0600204F0906104E0600214F0906633
:103CA3008FE0D394014003E014F0301B020568E574
:103CB30069D394644004D21C80020569E564D394FB
:103CC3000140021564D28ED0D0D082D083D0E032AE
:10101200C291C290D2B5C2217D027C007F071246E6
:101022000D8F45E545646060097D017F601245A82A
:10103200D221E4FDFC7F0B12460D8F45E54530E6DB
:10104200097D04E4FF1245CCD2217D017C007F079B
:1010520012460D8F45E5457008FD7FFF1245A8D267
:1010620021302103126000C288C2A8C2AA75890079
:101072001240FD90633FE0B4FA06A3E064CE607BC9
:10108200E4F54574372545F582E43463F583E4F0ED
:101092000545E545B443EC90633F74FAF0A374CE82
:1010A200F0A374CCF0906345740AF0E4A3F0A304B7
:1010B200F0A3F090633B74FFF0A3F0A3F0E4A3F07D
:1010C2009063567403F0E4F545E5452401FFE433EB
:1010D200FE74372545F582E43463F583E0FD12455D
:1010E200840545E545C3944340DFE4F5A775A61E94
:1010F20075A6E1907FF0F0A3F080FE90634A74033E
:10110200F0A374CCF0E4906349F090668CF0A3F005
:101112001236A6C2B51229A0C21C12437AD221C22B
:1011220023C2229065777408F09062B57424F0E4CB
:10113200A3F090633FE09062B7F0906340E090626A
:10114200B8F0906341E09062B9F0906342E090623F
:10115200BAF0906343E09062BBF0906344E0906227
:10116200BCF0756601E4906578F0C21DC21EC21F14
:10117200C220202118AF45FE7D0312378CE4FF12F6
:101182003B937E167F9AE4FBFDFC1232BC90668E86
:10119200E060037401F0E4906104F0F56890657614
:1011A200F0F56912464475A70775A61E75A6E1D229
:1011B200AFE4F569906104E0700312092190668F33
:1011C200E06401701D9080007410F09080A874FF9C
:1011D200F0A3F0A3F0A3F0E490668FF0D221C22234
:1011E200C223908008E0F54530E405D21D7410F06A
:1011F200E54530E508D21F9080087420F0E54530BF
:10120200E608D21E9080087440F0E568C39403405B
:1012120019908002E4F0908001F0908000F0E5687F
:1012220094064006E4F56812437A9080A0E07003C9
:101232001241F59080B8E0700312417B9080D0E0BB
:10124200700312431E908000E07013301D101233A1
:10125200C3906332EFF0D3940040031200369080C3
:1012620002E07006908000E06005D21B0211B3C25A
:101272001BE4F568906104E060030211B3202112BF
:10128200906579E0600C7E167F9C1235BEE4906515
:1012920079F0301F12123006906332EFF0D39400CF
:1012A2004005E0FF120032201E03021437122D0205
:1012B200906332EFF070030211B3906376E054BF93
:1012C200247F700302139214700302136A240260D3
:1012D200030213D92021077E167FA31235BE2025D3
:1012E2000302143790634EE07006906352E0606729
:1012F200906683E0FF90634EE0B50724906684E039
:10130200FE90634FE0B50618906685E0FE9063504C
:10131200E0B5060C906686E0FE906351E06E6037A1
:10132200906352E06F6003021437906684E0FF908E
:101332006353E06F6003021437906685E0FF9063A9
:1013420054E06F6003021437906686E0FF906355A5
:10135200E06F6003021437C2199065787401F012CD
:10136200467175660102143790668EE0600374015F
:10137200F090667BE0FF906378E06F6003021437C1
:1013820090667BE004F0E4F566906576F00214372F
:10139200301903021437906345E070030211B390D1
:1013A20062B4E06008906356741EF0800690635643
:1013B2007403F0124469D219E4F566906576F090F0
:1013C200668704F0E490667AF0A3F02021677E1627
:1013D2007FB11235BE805E90668EE060037401F0CC
:1013E200301952906376E020E74B906378E0FF90EB
:1013F200667AE0FE6F600D906682E07007EE146F11
:101402007033801390667AE004F0906332E0FFD389
:1014120094044003123AE19060007482F0A37401D4
:10142200F0906378E0906002F07E607F007D0312AE
:101432003DE60211B320190302155AE566706E12D9
:1014420044A5EF60237E647F76906477E02404FDF8
:10145200123DE6906682E07009906356E0F56602FE
:1014620011B3E4F5660211B3906687E0D3943C4071
:101472003C906682E070369062B4E070309066878D
:1014820004F0123948E4906476F0A37412F0906686
:101492007BE0906478F0A374FDF090610563A20193
:1014A20090647A63A2017F12122892809812465F9A
:1014B2008F45E545B401159060007483F0E4A3F014
:1014C2007E607F007D02123DE60211B3E545D394B2
:1014D20001401C9060007483F0A37401F0E5452480
:1014E200FEA3F07E607F007D03123DE60211B3E5AC
:1014F20066640160030211B3906576E004F0202176
:10150200077E167FBB1235BE906576E0FFD394014D
:10151200400B906356E0941E5003E004F0EFC39436
:1015220005400DC219E4906578F01246710211B3BC
:101532007C667D8390634AE0FAA3E0FB7F02123F60
:10154200777E647F76906477E02404FD123DE69016
:101552006356E0F5660211B3E566640160030211A9
:10156200B3906578E014604624FE60421470030272
:10157200164D240460030211B3E4F568202513908C
:1015820065787404F0906576E05401F075660102A6
:1015920011B39080027410F0E4906578F090657653
:1015A20004F075661290668374FFF00211B39066C0
:1015B20083E070030216379064767480F09064784A
:1015C2007401F0E4A3F0A304F0A37430F0A3747BDD
:1015D200F0E4F545747D2545F582E43464F58374C1
:1015E2007DF0747E2545F582E43464F583E4F0E50C
:1015F200452407906477F07C667D8390634AE0FA25
:10160200A3E0FB7F02123F777E647F76E5452409E3
:10161200FD123DE6906682E0601B124469D219E435
:10162200F566906576F090668704F0E490667AF04D
:10163200A3F00211B3302507E4906578F08006909C
:1016420065787404F07566120211B390800274100A
:10165200F0756603906576E06401FFF0906578743A
:1016620001F0EF7019906352E06013FCA3E0FDA358
:10167200E0FEA3E0FF90668312246C0211B3906334
:101682004EE0FCA3E0FDA3E0FEA3E0FF9066831220
:07169200246C0211B380FE7D
:01169900222E
:10003600906377E0B444047F0180027F009063768A
:10004600E0B447047E0180027E00EE5F604A906362
:100056003FE0906378F0906340E0906379F09063BE
:1000660041E090637AF0906342E090637BF09063A6
:1000760043E090637CF0906344E090637DF090638E
:10008600777452F09062AE63A2019080A863A201D9
:100096007F06122892020917906332E0C394085033
:1000A6000302092090633FE0FF906378E06F6003EE
:1000B600020920906340E0FF906379E06F600302DD
:1000C6000920906341E0FF90637AE06F60030209C4
:1000D60020906342E0FF90637BE06F60030209209B
:1000E600906343E0FF90637CE06F60030209209019
:1000F6006344E0FF90637DE06F6003020920906334
:1001060077E06444701A9080A8E0B4FF139062AE62
:1001160063A2019080A863A2017F06122892801034
:100126009062B2E09080ACF09062B3E09080ADF067
:1001360090668EE060037401F090668F7464F090B0
:1001460063777452F0906376E0646D60030202BADE
:100156007BFF7A1679C6121FD87BFF7A1679E09054
:10016600633FE0F54EA3E0F54FA3E0F550A3E0F5BD
:1001760051A3E0F552A3E0F553121FD8754EFF7553
:100186004F1775503D7551FF7552177553497BFFD3
:100196007A177916121FD87BFF7A177952121FD851
:1001A6007BFF7A1779B8121FD87BFF7A1779E5900B
:1001B6006345E0F54EA3E0F54FA3E0F550A3E0F567
:1001C60051121FD87BFF7A18790F90634EE0F54ED7
:1001D600A3E0F54FA3E0F550A3E0F551121FD87B3D
:1001E600FF7A18793D906352E0F54EA3E0F54FA3F0
:1001F600E0F550A3E0F551121FD87BFF7A18796B12
:1002060090633BE0F54EA3E0F54FA3E0F550A3E085
:10021600F551121FD87BFF7A18798E906337E0F577
:100226004EA3E0F54FA3E0F550A3E0F551121FD819
:100236007BFF7A1879AB121FD87BFF7A1879D4A284
:1002460025E433F54E121FD87BFF7A1979049066A0
:1002560082E0F54E121FD87BFF7A19792F90668EB1
:10026600E0F54E121FD87BFF7A1979629062B4E0EE
:10027600F54E121FD87BFF7A197994A217E433F54D
:100286004E121FD87BFF7A1979C090667CE0F54E36
:10029600A3E0F54FA3E0F550A3E0F551A3E0F55236
:1002A600A3E0F553121FD81231777BFF7A1A790B28
:1002B600121FD822906376E0644C70737E1A7F1109
:1002C600FBFDFC1232BC90637EE0F546A3E0F547E9
:1002D600E4F549E546906380F0A3E547F07E1A7F92
:1002E6004C7C637D807B021232BCE4F548854782F4
:1002F600854683E0FF74802548F582E43463F58300
:10030600EFF00547E547700205460548E548B41095
:10031600DC7E1A7F4F7C637D807B101232BC0549E0
:10032600E549C3941040AC7E1A7F521235BE229026
:100336006376E0646C7060F54A7E1A7F54FBFDFCC0
:100346001232BCE4F549E4906380F0A3E54AF07EFE
:100356001A7F4C7C637D807B021232BCE4F548A890
:100366004AE6FF74802548F582E43463F583EFF0AE
:10037600054A0548E548B410E67E1A7F4F7C637D42
:10038600807B101232BC0549E549C3940840B77E0C
:100396001A7F521235BE22906376E0644B7061F587
:1003A6004874682548F582E43463F583E060327466
:1003B600682548F582E43463F583E0F460237468C5
:1003C6002548F582E43463F583E0FF747E2548F51D
:1003D60082E43463F583E0B507100548E548B408C0
:1003E600C09061047432F00209179063767421F0AC
:1003F6003021030209177E1A7F8F1235BE020917B4
:10040600906376E0B4521A2021077E1A7F97123540
:10041600BE9063767472F07E637F767D08123D5FD0
:1004260022906376E0644970452021077E1A7FA2F8
:100436001235BE90637EE0F546A3E0F547E4F54845
:10044600854782854683E0FF74802548F582E4343B
:1004560063F583EFF00547E547700205460548E575
:1004660048B480DC7E637F767D8A123D5F2290638E
:1004760076E0644370462021077E1A7FAA1235BEB5
:1004860090637EE0F546A3E0F547E4F548854782AC
:10049600854683E493FF74802548F582E43463F54A
:1004A60083EFF00547E547700205460548E548B481
:1004B60080DB7E637F767D8A123D5F22906376E0E5
:1004C600645A70532021077E1A7FB31235BE90639B
:1004D6007EE0F546A3E0F5477C637D807B80AF47F1
:1004E600AE46124550E4F548854782854683E49337
:1004F600FF74802548F582E43463F583EFF0054701
:10050600E547700205460548E548B480DB7E637F13
:10051600767D8A123D5F22906376E0644460030232
:1005260005AE90637EE0FF64447003020917EFB4E2
:10053600310CC2217E1A7FBF1235BE0209179063A5
:100546007EE0B4300CD2217E1A7FCB1235BE020972
:100556001790637EE0B4320CD2227E1A7FD8123511
:10056600BE02091790637EE0B4330CC2227E1A7F66
:10057600E61235BE02091790637EE0B4340CD2232E
:100586007E1A7FF51235BE02091790637EE0B435F8
:100596000CC2237E1B7F021235BE02091790637EB2
:1005A600E0FF12001E020917906104E0701320217B
:1005B600077E1B7F101235BE9063767421F0020908
:1005C600179061047432F0906376E0FFB45104C270
:1005D600AF80FEEF645770452021077E1B7F1E12F9
:1005E60035BE90637FE0906332F0E4F54890633265
:1005F600E0FFE548C39F400302091774802548F5CC
:1006060082E43463F583E0FF90637EE0254824AD01
:10061600F582E43461F583EFF0054880D090637687
:10062600E0645360030206D12021077E1B7F291256
:1006360035BE90633FE0FF9061B6E06F703C90631B
:1006460040E0FF9061B7E06F7030906341E0FF904B
:1006560061B8E0B50724906342E0FF9061B9E0B568
:100666000718906343E0FF9061BAE0B5070C90630A
:1006760044E0FF9061BBE06F60169063767421F0F2
:100686003021030209177E1B7F381235BE02091777
:10069600E4F548E4F569AF48FE74AD2548F582E413
:1006A6003461F583E0FD1245840548E548C394FEB0
:1006B60040E1C2AFE4907FF0F0A3F0907FFD74AA12
:1006C600F0A374FFF0A37455F080FE906376E064A7
:1006D6004F705A90637EE0F546A3E0F547E547453F
:1006E60046700A2021077E1B7F411235BE20210756
:1006F6007E1B7F481235BEE4F54874802548F58296
:10070600E43463F583E0854782854683F00547E553
:1007160047700205460548E548B480DE90668DE0E0
:100726002480F090668CE03400F00209179063761E
:10073600E06445707490637EE0FEA3E0FF907FF076
:10074600EEF0A3EFF0D39400EE94044038907FF0DF
:10075600E0FEA3E0FF90668CE0FCA3E0FD9FEC9E2C
:100766004023E42FFFEE3401FED3ED9FEC9E50159F
:10077600C2AF907FFD74AAF0A374FFF0A37455F086
:10078600E4F5A780FE7E1B7F4A1235BE7BFF7A1BEF
:100796007952907FF0E0F54EA3E0F54F90668CE03D
:1007A600F550A3E0F551121FD8906376E0646560BA
:1007B6000302092090637EE0FFA3E0907FF0CFF074
:1007C600A3EFF0E4F546F547D3907FF1E095479027
:1007D6007FF0E095464020E4F5692547FFE546347D
:1007E60001FE854782854683E0FD1245840547E57F
:1007F600477002054680D17E1B7F5D123E6DEF4E2F
:100806006020120003906345EFF0120003906346E8
:10081600EFF0120003906347EFF012000390634875
:10082600EFF07E1B7F63123E6DEF4E6020120003D9
:1008360090634EEFF012000390634FEFF012000347
:10084600906350EFF0120003906351EFF07E1B7F30
:1008560069123E6DEF4E6020120003906352EFF076
:10086600120003906353EFF0120003906354EFF00D
:10087600120003906355EFF07E1B7F6F123E6DEF03
:100886004E602012000390633BEFF012000390636A
:100896003CEFF012000390633DEFF012000390630B
:1008A6003EEFF07E1B7F75123E6DEF4E602012000C
:1008B60003906337EFF0120003906338EFF01200F5
:1008C60003906339EFF012000390633AEFF0E4F51A
:1008D60048E4F569E5482401FFE433FE743725480A
:1008E600F582E43463F583E0FD1245840548E54866
:1008F600C3944340DCC2AFE4907FF0F0A3F0907F56
:10090600FD74AAF0A374FFF0A37455F0E4F5A78074
:0A091600FE7E637F767D08123D5FD0
:0109200022B4
:10451800AE07EEC39430400BEED394395005EE2429
:10452800D0FF22EEC39461400BEED394665005EEA3
:1045380024A9FF22EEC39441400BEED394465005C4
:08454800EE24C9FF22AF062298
:10462A009062ADE004F070069062ACE004F0906233
:0A463A00ACE0FEA3E0FF1245F02201
:1000030012462A124518EFC454F0FEC00612462ABF
:08001300124518D0E02FFF2276
:1042C100E4906B34F012462A906B35EFF0C39430D2
:1042D1004018E0FFD394395011906B34E02405F578
:1042E10082E43461F583EFF08011906B34E02405B2
:1042F100F582E43461F583E4F0800C906B34E004E2
:10430100F0E0D3940840BE754B00754C00754D002C
:0C431100E4F54E7B017A617905122B5E09
:01431D00227D
:043E6D008E4B8F4C9D
:103E71009062ACE4F0A374FFF012462AEF606EF496
:103E8100606B854C82854B83E493B507EC754D01DE
:103E9100E54C254DF582E4354BF583E4936025909F
:103EA10062ADE0254DFF9062ACE03400FE1245F0BA
:103EB100E54C254DF582E4354BF583E493B50704D4
:103EC100054D80CCE54C254DF582E4354BF583E479
:103ED1009370A6E54D24FFFFE434FFFE9062ADE050
:103EE1002FF09062ACE03EF07E007F0122E4FEFF05
:013EF10022AE
:1036A6007E1B7F7B123E6DEF4E70037F01227E1BD9
:1036B6007F7E123E6DEF4E600C12462AEF24D02418
:1036C600FF92258002D2257E1B7F84123E6DEF4E2F
:1036D600600C12462AEF24D0906682F08005E490B2
:1036E6006682F07E1B7F8A123E6DEF4E600C12469C
:1036F6002AEF24D090668EF08005E490668EF07EE8
:103706001B7F90123E6DEF4E600C12462AEF24D0BE
:1037160024FF92178002C2177E1B7F96123E6DEF22
:103726004E600C12462AEF24D09062B4F08005E475
:103736009062B4F090633F63A20190667C63A2013D
:103746007F0612289230173B7E1B7F9C123E6DEF40
:103756004E603012000390667CEFF0120003906614
:103766007DEFF012000390667EEFF0120003906684
:103776007FEFF0120003906680EFF0120003906670
:0637860081EFF07F00223C
:10442000906577E0C3947C40027F0A906577E0FE58
:1044300004F074B52EF582E43462F583EFF0BF0A20
:1044400027906577E0FF04F074B52FF582E43462BD
:10445000F583E4F0906577E0FF123EF290657774A3
:0944600008F09062B6E004F022BD
:10437A009080007480F090633763A201F583F58220
:10438A0063A2017F0812289290633F63A201908082
:10439A008863A2017F0A1228929080927407F0A380
:1043AA0074D0F0A37406F0906349E0FF9080B1F0F6
:1043BA009080E1EFF09080957455F0A3F090800022
:0A43CA007401F090800974F0F022F5
:1041F500908009E04410F09080A0E070609080A16C
:104205007482F09080A874FFF0A3F0A3F0A3F07F70
:10421500039080AEEFF0A374CBF09080007402F0B1
:10422500906B2312247800000000906B23E09080AF
:1042350040F0906B24E0908041F0906B25E09080F9
:1042450042F0906B26E0908043F0A3E4F0A3F0A346
:0D425500F0A3F0908018F0A3F0A3F0A3F008
:014262002239
:10431E00908009E04440F09080D17482F07F039049
:10432E0080DEEFF0A374CCF09080027402F0906BFC
:10433E002712247800000000906B27E0908058F040
:10434E00906B28E0908059F0906B29E090805AF0A5
:10435E00906B2AE090805BF0A3E4F0A3F0A3F0A3AF
:0B436E00F0908030F0A3F0A3F0A3F06B
:014379002221
:10417B00908009E04420F09080B8E0706C9080B99A
:10418B007482F07F039080C6EFF07FCDA3EFF07FBA
:10419B00039080C4EFF0A374CDF09080C074FFF057
:1041AB00A3F0A3F0A3F09080017402F0906B2B129C
:1041BB00247800000000906B2BE090804CF0906B0B
:1041CB002CE090804DF0906B2DE090804EF0906B3A
:1041DB002EE090804FF0A3E4F0A3F0A3F0A3F090B7
:0941EB008024F0A3F0A3F0A3F07E
:0141F40022A8
:103F77008C468D47A907EAFDE975F018A424ACFF24
:103F8700E5F034808F82F583EDF0EBFDE975F018ED
:103F9700A4FFAEF024ACFBEE34808B82F583A3ED57
:103FA700F08547828C83E0FDEF24A8FFEE3480FE86
:103FB7008F82F583EDF08547828C83A3E08F828E15
:103FC70083A3F0854782854683A3A3E0FDE975F0C7
:103FD70018A424A8FFE5F03480FE8F82F583A3A3FD
:103FE700EDF08547828C83A3A3A3E08F828E83A302
:043FF700A3A3F0226E
:063D5F008D4BAB07AA0624
:103D6500908000E030E5079065797401F022906B52
:103D750023E0FCA3E0FDA3E0FEA3E0F54F8E4E8D0E
:103D85004D8C4CAE02AF038E838F8263A201E54E4C
:103D9500540744C0F583854F8263A201AF4B1229B6
:103DA50004E4FCFDFEE54F254BF54FEE354EF54E93
:103DB500ED354DF54DEC354CF54C908040E54CF02E
:103DC500A3E54DF0A3E54EF0A3E54FF09080007418
:103DD50020F0AF4FAE4EAD4DAC4C906B2312246C22
:013DE50022BB
:063DE6008D46AB07AA06A2
:103DEC00908002E030E5079065797403F022906BC7
:103DFC0027E0FCA3E0FDA3E0FEA3E0F54A8E498D8D
:103E0C00488C47AE02AF038E838F8263A201E549D3
:103E1C00540744D0F583854A8263A201AF46122928
:103E2C0004E4FCFDFEE54A2546F54AEE3549F54924
:103E3C00ED3548F548EC3547F547908058E547F0A7
:103E4C00A3E548F0A3E549F0A3E54AF0908002749D
:103E5C0020F0AF4AAE49AD48AC47906B2712246CAA
:013E6C002233
:023B93008F465B
:103B9500908001E030E5099065797402F07F00229C
:103BA500906B2BE0FCA3E0FDA3E0FEA3E0F54A8EBD
:103BB500498D488C4790667C63A201E549540744CA
:103BC500C8F583854A8263A2017F0612291AE54A50
:103BD5002406F54AE43549F549E43548F548E43520
:103BE50047F54790657A63A201E549540744C8F54E
:103BF50083854A8263A201AF4612291AE4FCFDFEC1
:103C0500E54A2546F54AEE3549F549ED3548F54885
:103C1500EC3547F54790804CE547F0A3E548F0A320
:103C2500E549F0A3E54AF09080017420F0AF4AAE73
:0D3C350049AD48AC47906B2B12246CAF4694
:013C4200225F
:1033C3009081E0E0F5460546054605460546054677
:1033D30005460546054605460546908010E0F54935
:1033E300A3E0F54AA3E0F54BA3E0F54C9081E1E0BF
:1033F300F546054605460546054605460546054682
:10340300054605460546908014E0F54DA3E0F54ECC
:10341300A3E0F54FA3E0F550E54FB54B08E550B5F4
:103423004C037F0022E4F546E54F540744E0F5835F
:1034330085508263A20190637663A2017F081229FB
:103443004A90637863A2019062AE63A2017F061281
:103453002892906376E0F547A3E0F548E4F54690BB
:103463006376E0702AA3E024F8F546E54F54074459
:10347300E0F58385508274082582F582E43583F56F
:103483008363A20190637663A201AF4612294AAE19
:1034930047E4FCFDE5502548F550E54F3EF54FED7B
:1034A300354EF54EEC354DF54D908014E54DF0A3BA
:1034B300E54EF0A3E54FF0A3E550F0908000744093
:0334C300F0AF4621
:0134C60022E3
:102D02009081E6E0F5460546054605460546054638
:102D120005460546054605460546908028E0F549E4
:102D2200A3E0F54AA3E0F54BA3E0F54C9081E7E080
:102D3200F546054605460546054605460546054649
:102D420005460546054690802CE0F54DA3E0F54E7C
:102D5200A3E0F54FA3E0F550E4F546E54FB54B0A85
:102D6200E550B54C05C21E022E6EE54F540744F0E5
:102D7200F58385508263A20190637663A2017F0886
:102D820012294A906376E0F547A3E0F548E5484505
:102D92004770099080027410F07F0022906683E0F1
:102DA200FFF46030906378E06F6003022E35906626
:102DB20084E0FF906379E06F7079906685E0FF9020
:102DC200637AE06F706D906686E0FF90637BE06FE0
:102DD2006031805F906378E0906683F0906379E081
:102DE200906684F090637AE0906685F090637BE071
:102DF200906686F090637CE0FFA3E090634ACFF098
:102E0200A3EFF0906376E0702AA3E024F8F546E59C
:102E12004F540744F0F58385508274082582F58269
:102E2200E43583F58363A20190637663A201AF4622
:102E320012294AAE47E4FCFDE5502548F550E54F1E
:102E42003EF54FED354EF54EEC354DF54DAF4CAEF2
:102E52004BAD4AAC49AB50AA4FA94EA84DD3122450
:102E62005B40099080027410F07F002290802CE574
:102E72004DF0A3E54EF0A3E54FF0A3E550F09080AE
:062E8200027440F0AF46AF
:012E88002227
:103006009081E3E0F5460546054605460546054634
:103016000546054605460546054690801CE0F549E9
:10302600A3E0F54AA3E0F54BA3E0F54C9081E4E07C
:10303600F546054605460546054605460546054642
:10304600054605460546908020E0F54DA3E0F54E81
:10305600A3E0F54FA3E0F550E4F546E54FB54B0A7E
:10306600E550B54C05C21F02315CE54F540744E8F4
:10307600F58385508263A20190600463A2017F0EEE
:10308600122960906004E0F547A3E0F54890600CD3
:10309600E0FFF4604A90667CE0FEEF6E7079A3E094
:1030A600FF90600DE06F706F90667EE0FF90600E9F
:1030B600E06F706390667FE0FF90600FE06F70577F
:1030C600906680E0FF906010E06F704B906681E044
:1030D600FF906011E06F703FE4906013F0800890FD
:1030E600601374FFF0D2D9906004E0702AA3E02444
:1030F600F2F546E54F540744E8F583855082740E91
:103106002582F582E43583F58363A201906004632A
:10311600A201AF46122960AE47E4FCFDE550254802
:10312600F550E54F3EF54FED354EF54EEC354DF588
:103136004DAF4CAE4BAD4AAC49AB50AA4FA94EA8C9
:103146004DD312245B5006E548454770099080012F
:103156007410F07F0022908020E54DF0A3E54EF03C
:10316600A3E54FF0A3E550F09080017440F0AF4620
:013176002236
:0435BE008E4B8F4C55
:1035C200908000E030E5079065797401F022906BFD
:1035D20023E0FCA3E0FDA3E0FEA3E0F5528E518DB3
:1035E200508C4FE552FFE5515407FEE42FF54EEEA5
:1035F20034C0F54D854E82F5837423F0054EE54EB9
:103602007002054D534DC7F582854D83740AF0054E
:103612004EE54E7002054D534DC790633F63A201C4
:10362200854D83854E8263A2017F061229047406AA
:10363200254EF54EE4354DF54D854B83854C826321
:10364200A201854D83854E8263A2011228E8E4FC23
:10365200FDFE906B23E0F8A3E0F9A3E0FAA3E02FCC
:10366200FFEE3AFEED39FDEC38FCEF2408FFE43EB4
:10367200FEE43DFDE43CFC906B2312246C906B2332
:10368200E0908040F0906B24E0908041F0906B25B8
:10369200E0908042F0906B26E0908043F0908000B2
:0336A2007420F0A1
:0136A5002202
:0A32BC008E4D8F4E8C4F8D508B51BC
:1032C600908000E030E5079065797401F022906BFC
:1032D60023E0FCA3E0FDA3E0FEA3E0F5578E568DA8
:1032E600558C54E557FFE5565407FEE42FF553EE8B
:1032F60034C0F552855382F5837423F00553E553A4
:10330600700205525352C7F582855283740AF0053E
:1033160053E553700205525352C790633F63A201AF
:1033260085528385538263A2017F0612290474069F
:103336002553F553E43552F552854D83854E826308
:10334600A20185528385538263A2011228E88F5811
:10335600EF2553F553E43552F552E5516017854F85
:103366008385508263A20185528385538263A201BD
:10337600AF51122904E55824082551F551FFE4FC04
:10338600FDFEE5572FF557EE3556F556ED3555F555
:1033960055EC3554F554908040E554F0A3E555F0CE
:1033A600A3E556F0A3E557F09080007420F0AF57E0
:0C33B600AE56AD55AC54906B2312246C45
:0133C20022E8
:06386D008E478F488D49D3
:10387300908000E030E5079065797401F022906B49
:1038830023E0FCA3E0FDA3E0FEA3E0F54F8E4E8D05
:103893004D8C4CE54FFFE54E5407FEE42FF54BEE00
:1038A30034C0F54A854B82F5837423F0054BE54B11
:1038B3007002054A534AC7F582854A83EBF0054BEC
:1038C300E54B7002054A534AC790633F63A20185E3
:1038D3004A83854B8263A2017F061229047406255D
:1038E3004BF54BE4354AF54A85478385488263A205
:1038F30001854A83854B8263A201AF49122904746F
:10390300082549F549FFE4FCFDFEE54F2FF54FEE91
:10391300354EF54EED354DF54DEC354CF54C90806F
:1039230040E54CF0A3E54DF0A3E54EF0A3E54FF0E1
:103933009080007420F0AF4FAE4EAD4DAC4C906B09
:043943002312246CBB
:01394700225D
:023EF2008F5FE0
:103EF400908000E030E5079065797401F022906BC2
:103F040023E0FCA3E0FDA3E0FEA3E0F5638E628D55
:103F1400618C60E563FFE5625407FEE42FFFEE3435
:103F2400C09062B563A201F5838F8263A201AF5F83
:103F3400122904E4FCFDFEE563255FF563EE3562BA
:103F4400F562ED3561F561EC3560F560908040E532
:103F540060F0A3E561F0A3E562F0A3E563F090806F
:103F6400007420F0AF63AE62AD61AC60906B23125D
:023F7400246CBB
:013F76002228
:06378C008E468F47AB05DD
:10379200908000E030E5079065797401F022906B2B
:1037A20023E0FCA3E0FDA3E0FEA3E0F54D8E4C8DEB
:1037B2004B8C4AE54DFFE54C5407FEE42FF549EEEC
:1037C20034C0F548854982F5837423F00549E549FB
:1037D200700205485348C7F582854883EBF00549D6
:1037E200E5497002054890633F63A20185488385DD
:1037F200498263A2017F0612290474062549F5490C
:10380200E43548F5485348C7E546854982854883EB
:10381200F00549E549700205485348C7F5828548D5
:1038220083E547F00549E549700205485348C7E575
:103832004D240AF54DE4354CF54CE4354BF54BE49B
:10384200354AF54A908040E54AF0A3E54BF0A3E5FE
:103852004CF0A3E54DF09080007420F0AF4DAE4CDB
:0A386200AD4BAC4A906B2312246CAE
:01386C002239
:0A465400E4FEEEC39F50030E80F851
:01465E002239
:1045F000A2AF9226C2AF438E2075D2028F828E83E5
:0C460000E0FFE4F5D2538EDFA22692AF5B
:01460C00228B
:10458400E5D220E0FBA2AF9226C2AF43D2028F82D3
:104594008E83EDF075D25063D250A22692AFE5D24D
:0345A40020E0FB19
:0145A70022F1
:1040FD00E4FDED2401FFE433FE1245F074372DF598
:10410D0082E43463F583EFF00DBD3FE6E4FDED246D
:10411D007FFFE433FE1245F0742D2DF582E43461FA
:10412D00F583EFF0742D2DF582E43461F583E070A5
:10413D001B742D2DF582E43461F5837420F0742EFB
:10414D002DF582E43461F583E4F080040DBD80BE6D
:10415D00E49061ACF0FDEDFF7E001245F074AD2DE5
:0D416D00F582E43461F583EFF00DBDFEE94D
:01417A002222
:024550008B4B93
:10455200A2AF9226C2AF85A24C53A2FE8E838F8257
:1045620005A28C838D82740912298EE54B53A2FE1B
:1045720043A22012299053A2DF854CA2A22692AF19
:01458200FF39
:014583002215
:10460D00A2AF9226C2AF8C838D82EF12298E43A268
:0C461D002012299053A2DFA22692AFFFCA
:01462900226E
:0245A8008F463C
:1045AA00A2AF9226C2AFE4F5838D82740612298ED9
:1045BA00E54643A22012299053A2DFA22692AF7F9A
:0145CA0001EF
:0145CB0022CD
:0245CC008F4618
:1045CE00A2AF9226C2AFE4F5838D82740A12298EB1
:1045DE00E54643A22012299053A2DFA22692AF7F76
:0145EE0001CB
:0145EF0022A9
:1027B700A907E7FFA805EF93C3966008403B74FCA1
:1027C7002FFF80F00F08EF93C3966008402B74FB30
:1027D7002FFF80E00F08EF93C3966008401B74FA41
:1027E7002FFF80D00F08EF93D3966008400B74F942
:1027F7002FFF80C01F1F1F1F1FEF54FEF80303F793
:10280700E893FC08E893FD08E893FE08E893FF22A5
:1028170009E993C39D6008402974FB29F980F109F0
:10282700E993C39E6008401A74FA29F980E209E91E
:1028370093D39F6008400B74F929F980D3191919AC
:102847001919E9C313C313FF22740093F8ECC39853
:102857004024701F740193F8EDC3984019701474E5
:0E2867000293F8EEC398400E7009740393F8C4
:10287500EFC39840037F00227F0122EDF8E6F008C0
:10288500A3DFFA22EDF8E0F608A3DFFA22E0A3635E
:10289500A201F0A363A201DFF475A2002263A201E5
:1028A500F0A363A20122E0A363A201F0A363A20146
:1028B500E0A363A201F0A363A201E463A201F0A374
:1028C50063A201DFE175A20022E0A363A2016DFE10
:1028D500936CFDEE058393FC158363A201DFEA7516
:1028E500A200227F00E493A363A201F00F600CA372
:1028F500E583C2E3F58363A20180EA75A20022E0C5
:10290500A363A201F0A3E583C2E3F58363A201DF1C
:10291500EE75A20022E0A363A201F0A3E583C2E461
:10292500D2E3F58363A201DFEC75A20022E0A36385
:10293500A201F0A3E58344F8C2E5F58363A201DFB4
:10294500EC75A20022E583C2E3F583E0A363A2014F
:10295500F0A363A201DFEE75A20022E583C2E4D2F3
:0A296500E3F583E0A363A201F0A3F1
:10296F0063A201DFEC75A20022E58344F8F583E052
:10297F00A363A201F0A363A201DFEE75A20022F907
:10298F0022C002C004C00612FFF0D006D004D0024D
:01299F002215
:10001E00BF360BD209E4F526F527F542F543BF3777
:04002E0002C20922DF
:10426300C2A9438902906B1EE0FFF58C8F8A75D932
:104273000475DA4875DB3175DC4975DD4975DE3166
:10428300E4F5E9F5F9F5EBF5FB906B1CE0601675C9
:10429300EC1075ED10E4F5FCF5FD753E08753C106A
:1042A300753D01801375EC8075ED80E4F5FCF5FD3B
:0E42B300753E80F53C753D10E4F5EEF5FE22FB
:1044DF00E4FEAF8CEFFD906B1DE07003A3E06D6009
:1044EF00051242637E01E5D920E2057E0212426386
:1044FF00E58920E1051242637E03D28C75D84075A1
:08450F00B740D2AED2AFAF06F7
:014517002281
:03003300022E8911
:0B2E8900C0E0C083C082C0D075D0083C
:102E9400C2AF30DC56C3E5EC95EEC3953E5012E567
:102EA4003D25ECF5EC30D70405FC801685FCFC8050
:102EB40011C3E5EC953DF5EC30D70415FC80038592
:102EC400FCFC300924852782852683E590F00527BC
:102ED400E52770020526F582852683E5EEF00527B1
:102EE400E5277002052653260FC2DC30D9293009A4
:102EF40024852782852683E590F00527E52770023F
:102F04000526F582852683E5EBF00527E527700283
:102F1400052653260FC2D930DA69E53C700405FC56
:102F24008010E53C25ECF5EC30D70405FC800385E6
:102F3400FCFC300A4CE5285480FFE52825E0F52800
:102F44003097020528200803632801302F19E5284B
:102F540054E06544702BEF7028753F08F53A8528D6
:102F64002BF528C22F801A053FE53F5407701253F2
:102F74003F3FE53F131313541F242AF8A62875284E
:102F840000C2DA30DB71E53C700405FD8010E53CDD
:102F940025EDF5ED30D70405FD800385FDFDE54005
:102FA400653B6029E53B54077013E53B1313135449
:102FB4001F2432F8E6F5292007036329FFE52933A6
:102FC4009296E52925E0F529053B533B3FB2923023
:102FD4000923852782852683E590F00527E5277058
:102FE400020526F582852683E4F00527E52770028D
:092FF400052653260FC2DBD2AF03
:092FFD00D0D0D082D083D0E032A4
:101BA2003E2A2C312CCFE0F0E0ECE5F2F0FB20F104
:101BB200E8EDF5F0EEEDEDEEE3EE20EFEEF0F2E023
:101BC2000A003E4C2C4230312C256C752CD1EAEEA9
:101BD200F0EEF1F2FC20EEE1ECE5EDE02C35302CFC
:101BE2003130302C3230302C3330302C3630302CF7
:101BF200313230302C323430302C343830300A002C
:101C02003E422C4731302C2562752CC8EDE2E5F0BE
:101C1200F1E8FF20EDE020EFF0E8B8ECE50A003E45
:101C2200422C4731312C2562752CC8EDE2E5F0F1EA
:101C3200E8FF20EDE020EFE5F0E5E4E0F7E50A005B
:101C42003E422C4730322C2562752CD3EFF0E0E275
:101C5200EBE5EDE8E520EFEEF2EEEAEEEC202028EF
:101C62005254532D435453290A003E532C473033C8
:101C72002C256C752CC7E0E4E5F0E6EAE020F1F2F1
:101C8200E0F0F2E020EFE5F0E5E4E0F7E828ECF13F
:101C9200290A003E532C4730332C256C752C202A00
:101CA200E7E0E4E5F0E6EAE020F1F2E0F0F2E0203D
:101CB200EFE5F0E5E4E0F7E828ECF1290A003E530D
:101CC2002C4732302C256C752CC2F0E5ECFF20EE4F
:101CD200E6E8E4E0EDE8FF20EEF2E2E5F2E028ECEF
:101CE200F1290A003E2A2C312CC0E4E0EFF2E5F0A3
:101CF20020F1E8EDF5F0EEEDEDEEE3EE20EAE0EDB9
:101D0200E0EBE02E20CFF0EEF2EEEAEEEB20D2CCCA
:101D12003132300A003E422C4B30342C2562752C75
:101D2200D0E5E6E8EC20EFF0EEF1EBF3F8EAE8209C
:101D3200EAE0EDE0EBE020F1E2FFE7E80A003E53E3
:101D42002C4B30312C25732CD1EFE8F1EEEA20CA6E
:101D5200CF0A003E532C4B30322C25732CCAEEEBAB
:101D62002DE2EE20E3F0F3EFEF20D2C8D20A003EDC
:101D7200532C4B30332C25732CCFF0E8EEF0E8F2E5
:101D8200E5F220CED220EA20C7C3D2C8D20A003C54
:101D920021003C4230313D003C4731303D003C4760
:101DA20031313D003C4730323D003C4730333D004D
:101DB2003C4732303D003C4B30343D003C4B3031EF
:101DC2003D003C4B30323D003C4B30333D000ACFAE
:101DD200EEEFFBF2EAE020EEF2EFF0E0E2EAE820DA
:101DE200F1EBE8F8EAEEEC20E4EBE8EDEDEEE3EE01
:101DF20020EFE0EAE5F2E021000ACEF2EFF0E0E2C5
:101E0200EAE020D2D30A000ACEF2EFF0E0E2EAE002
:101E120020E7E0EFF0EEF1E020EEF220F1E5F0E273
:101E2200E5F0E00A000A435243206572726F7221A4
:101E32002020000ACFF0E8B8EC20E8EDF4EEF0EC58
:101E4200E0F6E8E82020000AD7F3E6EEE920CACF60
:101E5200212020000AC6E4E0EB20E8EDF4F320E0C4
:101E620020F2F3F220F7F2EE2DF2EE20EDE520F271
:101E7200EE2E2E2E000ACAE2E8F2E0EDF6E8FF208E
:101E8200D2D3212020000AC6E4E0EB20EAE2E8F205
:101E9200E0EDF6E8FE20D2D32C20E020F2F3F2208F
:101EA200F7F2EE2DF2EE20E4EBE8EDEDEEE52E2E6C
:101EB2002E2020000ACDE5F220E8EDF4EEF0ECE071
:101EC200F6E8E8212020000ACFF0E8B8EC20E7E0AD
:101ED200EFF0EEF1E02020000ACDE0F7E0EBEE209B
:101EE200EFF0E8B8ECE0000AC8F1F2E5EAEBEE2028
:101EF200E2F0E5ECFF20EEE6E8E4E0EDE8FF20EEBC
:101F0200F2E2E5F2E0000AC7E0EFF0EEF120E3F0E2
:101F1200F3EFEFFB20D2C8D2200020EEF220CACF8E
:101F220020000A000ACEF2EFF0E0E2EAE020CED290
:101F320020EDE020CACF2000202020CFEEE2F2EEFA
:101F4200F020EAEEECE0EDE4FB0A000D0AC8F1F243
:101F5200E5EAEBEE20E2F0E5ECFF20EEE6E8E4E075
:101F6200EDE8FF20E4EEF1F2E0E2EAE820EFE0EA59
:041F7200E5F2E000B4
:103A27005266900000000000000000000000000047
:103A3700000000000060A06A740005000200000595
:103A4700000200000500020000050002000005005A
:103A57000200000500020000050002000005000248
:103A6700000005000200000500020000050002003A
:103A7700000500020000050002000005000200002A
:103A87000500020000050002000005000200000515
:103A9700000200000500020000050002000005000A
:103AA70002000005000200000500020000050002F8
:103AB70000000500020000050002000005000200EA
:103AC70000050002000005000200000500020000DA
:093AD700050002000005000200D8
:0100320022AB
:103177007BFF7A1B79A2121FD8906B1CE0602FA3EC
:10318700E0FEA3E0FFC3E49FFFE49EFEAB07FAE483
:10319700F9F8FF7EC27D01FC1223BB8F518E508D43
:1031A7004F8C4E7BFF7A1B79C4121FD8802F906BF0
:1031B7001DE0FEA3E0FFC3E49FFFE49EFEAB07FA1A
:1031C700E4F9F87F207E1CFDFC1223BB8F518E5043
:1031D7008D4F8C4E7BFF7A1B79C4121FD87BFF7AE9
:1031E7001C7902A208E433F54E121FD87BFF7A1C24
:1031F7007921A207E433F54E121FD87BFF7A1C7999
:1032070042A20CE433F54E121FD8300C1F7BFF7A15
:103217001C796C906723E075F00AA4FFAEF0E48F89
:10322700518E50F54FF54E121FD8801D7BFF7A1C2B
:103237007995906723E075F00AA4FFAEF0E48F510B
:103247008E50F54FF54E121FD87BFF7A1C79C09030
:1032570067C8E075F00AA4FFAEF0E48F518E50F511
:103267004FF54E121FD87BFF7A1C79E6121FD87BC9
:10327700FF7A1D7917A213E433F54E121FD8754E46
:1032870001754F677550247BFF7A1D7940121FD84F
:10329700754E01754F687550C97BFF7A1D795512B8
:1032A7001FD8754E01754F667550A27BFF7A1D7941
:0532B70071121FD82276
:023FFB008D48EF
:103FFD00AA06A907754B018A4C894DE4F54912466D
:10400D002A8F4AE54A643C6030E54A642C602AAB4D
:10401D004BAA4CA94DE54A12234B7401254DF54D84
:10402D00E4354CF54C054912462A8F4AE54A643C65
:10403D006007E549C3954840D6E5497016AB4BAAD4
:10404D004CA94D742012234B7401254DF54DE435CB
:10405D004CF54CE549B5480C74FF254DF54D74FFF5
:0E406D00354CF54CAB4BAA4CA94DE412234B3D
:01407B002222
:102598007E1D7F91123E6DEF4E70037F01227E1DDE
:1025A8007F94123E6DEF4E700302263F1242C19097
:1025B8006B3012246CE4FFFEFDFC906B30E0F8A356
:1025C800E0F9A3E0FAA3E0FBC312245B6025906B5B
:1025D80030E0F8A3E0A3E0A3E0E47F207E1CFDFC4C
:1025E8001223BB12244D906B1DEEF0A3EFF0E49084
:1025F8006B1CF0E47FB07E04FDFC906B30E0F8A328
:10260800E0F9A3E0FAA3E0FBD312245B4038906B17
:102618001C7401F0906B30E0F8A3E0A3E0A3E07F26
:10262800007EC27D017C001223BB12244D906B1DDD
:10263800EEF0A3EFF0800F906B1D74FFF0A374B859
:10264800F0E4906B1CF07E1D7F9A123E6DEF4E6099
:102658000C12462AEF24D024FF92088002C2087E7A
:102668001D7FA0123E6DEF4E600C12462AEF24D05B
:1026780024FF92078002C2077E1D7FA6123E6DEFDF
:102688004E600C12462AEF24D024FF920C8002C21E
:102698000C7E1D7FAC123E6DEF4E60131242C1E4FA
:1026A8007B0AFAF9F81223BB906723EFF08005E460
:1026B800906723F07E1D7FB2123E6DEF4E601112BF
:1026C80042C1E47B0AFAF9F81223BB9067C8EFF01D
:1026D8009067C8E07003740AF07E1D7FB8123E6DE3
:1026E800EF4E600C12462AEF24D024FF921380028A
:1026F800C213E4906B2FF07E1D7FBE123E6DEF4E2D
:10270800600B7E677F247D80123FFB8023906B2FB8
:10271800E0FF04F074242FF582E43467F583742015
:10272800F0906B2FE02424F582E43467F583E4F01D
:10273800E4906B2FF07E1D7FC4123E6DEF4E600B50
:102748007E687FC97D80123FFB8023906B2FE0FF5E
:1027580004F074C92FF582E43468F5837420F0908E
:102768006B2FE024C9F582E43468F583E4F0E49043
:102778006B2FF07E1D7FCA123E6DEF4E600B7E669A
:102788007FA27D80123FFB8023906B2FE0FF04F037
:1027980074A22FF582E43466F5837420F0906B2FD1
:0E27A800E024A2F582E43466F583E4F07F00BD
:0127B6002200
:1044A500301234E4906476F0906A72E0FD9064779F
:1044B500F090667BE0906478F0A37404F0906972E4
:1044C500E0543FF063A20190647A63A201AF051244
:0A44D5002892C2127F01227F00220C
:1029A000906B1D74FFF0A374B8F0E4906B1CF09072
:1029B00067C87464F0E4906B19F0C210122598E4B3
:1029C000F547F54674242546F582E43467F583E03F
:1029D000FF6070E547C394205069EFB420040546BA
:1029E00080E2E54775F005A42474F9746A35F0FABD
:1029F000906B157401F0A3EAF0A3E9F07424254666
:102A0000F9E43467FA7B01C0031B8B4B754C0075EE
:102A10004D00E4F54ED003122B5E906B15E0FBA346
:102A2000E0FAA3E0F9EF12234B054774242546F59D
:102A300082E43467F583E0FF64206088EF608505F9
:102A40004680E8E5477005D210022B5AE4F547F5B9
:102A50004674C92546F582E43468F583E0FF607367
:102A6000E547C39420506CEFB42004054680E2E5AE
:102A70004775F005A42474F9746A35F0FA906B1563
:102A80007401F0A3EAF0A3E9F074C92546F9E4342F
:102A900068FA7B01C0031B8B4B754C00754D00E43D
:102AA000F54ED003122B5E906B15E0FBA3E0FAA36A
:102AB000E0F9900003EF12235D054774C92546F540
:102AC00082E43468F583E0FF64206085EF6082056E
:102AD0004680E8E4F547F54674A22546F582E434DD
:102AE00066F583E0FF6073E547C39420506CEFB454
:102AF0002004054680E2E54775F005A42474F974C6
:102B00006A35F0FA906B157401F0A3EAF0A3E9F0CE
:102B100074A22546F9E43466FA7B01C0031B8B4B93
:102B2000754C00754D00E4F54ED003122B5E906B92
:102B300015E0FBA3E0FAA3E0F9900001EF12235D9A
:102B4000054774A22546F582E43466F583E0FF6408
:0D2B5000206085EF6082054680E812426338
:012B5D002255
:104469007544C0C209C206E4F528C212C20FC201CE
:10447900D211F53AF53F906B1AF09067C7F03013F7
:10448900129067227403F0D22F9067C8E09067C733
:0C449900F08005E4906722F01244DF225E
:10407C00AC07D227E4FE9067A4E0FD25E0F0EC301D
:10408C00E709E04401F0A227B392270517E517B41E
:10409C00081C9067A4E0851682851583F00516E54B
:1040AC001670020515906A73E004F0E4F517EC2520
:1040BC00E0FC0EBE08C09067A4E0FF25E0F0A2264D
:1040CC00302701B350079067A4E04401F00517E5D1
:1040DC0017B4081C9067A4E0851682851583F0053B
:1040EC0016E51670020515906A73E004F0E4F517F6
:0140FC0022A1
:0234C700AB0751
:1034C900E4FD200038906B14E0FF30E10A6402F05B
:1034D900906B18E06429F0906B14E0FF25E0F09000
:1034E9006B18E0FE30E707906B14E04401F0EE251D
:1034F900E0906B18F0EB30E704E04401F00517E5C4
:103509001724F8601F1460468000EB30E70A431B5C
:1035190001A204B392048003531BFEE51B25E0F5C9
:103529001B0235AEEB30E70A431B01A204B3920438
:103539008003531BFE851482851383E51BF0051454
:10354900E51470020513906A72E004F080573005A3
:1035590026D20E300D1E906B14E0FF30E10A640292
:10356900F0906B18E06429F0906B18E0FF906B14F1
:10357900E04FFF227F0022300413EB20E720D20521
:10358900E51BB42004D20D8015C20D8011EB30E784
:103599000DD205E51BB42004D20D8002C20DC20074
:1035A900D204E4F517EB25E0FB0DED640860030296
:0435B90034CB7F0090
:0135BD0022EB
:0243D400AB0735
:1043D600E4906A73F075476975484A7515697516EC
:1043E600F2854882854783E044C0F0E4F517FAEA8F
:1043F600C39B5018854882854783E0FFC22612403A
:104406007C0548E548700205470A80E3D226E4FFAA
:0944160012407C7515697516F25F
:01441F00227A
:023AE1008F460E
:103AE300300103023B9274FC2546F546131313542D
:103AF3001FFF2546FFE433CF2402CF3400FEC3EF7C
:103B03009420EE64809480401130230B7E1D7FD07F
:103B1300E4FBFDFC1232BCD2112275490185154A22
:103B230085164B906A73E0FBE4F075476375487A3A
:103B33007515677516A6854882854783E044C0F0EE
:103B430085174CE4F5171546FAEAC39546501885D0
:103B53004882854783E0FFC22612407C0548E5483A
:103B6300700205470A80E2D226E4FF12407CD201AC
:103B7300906A73E09067C6F0906A73EBF0854A151C
:0F3B8300854B16751801751967751AA6854C17AD
:013B92002210
:10394800E4FF0F2405F582E43461F5837405F00F74
:1039580074052401F582E43461F583E4F0754601C9
:10396800754766754895FEAB46E5481548AA477001
:10397800021547F91222D2FDAC070F74052CF58207
:10398800E43461F583EDF00EBE04DC75460175473D
:1039980066754899E4FEAB46E5481548AA477002A3
:1039A8001547F91222D2FDAC070F74052CF582E4F5
:1039B8003461F583EDF00EBE04DC7546017547668B
:1039C80075489DE4FEAB46E5481548AA47700215C0
:1039D80047F91222D2FDAC070F74052CF582E434A6
:1039E80061F583EDF00EBE04DC754601754766751A
:1039F80048A1E4FEAB46E5481548AA4770021547BA
:103A0800F91222D2FDAC070F74052CF582E434615B
:083A1800F583EDF00EBE04DCA5
:013A20002283
:07466A00C20EC206C20522C8
:1009210030092DC3E5279543FFE5269542FED3EF18
:100931009440EE940040197B087D40AF43AE4212D3
:10094100386DE5432440FFE43542540FF5428F43AF
:1009510020190302101130180AC2189067C7E0600D
:100961000214F0906722E0B40800501F900974F857
:10097100282873020992020A6D020A6D020B6E02A7
:100981000E3A020B6E020FC3020FEFE4906722F0E2
:10099100223013139067227403F0D22F9067C8E0BE
:1009A1009067C7F0D20A22200103020A669067C647
:1009B100E0906A73F0C201D214E4F546906A73E0E4
:1009C100FFE546C39F5026AB18AA19A91A1222D2D5
:1009D100FE744A2546F582E43469F583EEF074012C
:1009E100251AF51AE43519F519054680CF751569EB
:1009F10075164A8515118516128F10851682851573
:100A010083A3E05478FF64706003BF3825906722A8
:100A11007401F09067A57406F0D20320230302103D
:100A2100117E1D7FFB906A73E0FBAD16AC1512328F
:100A3100BC223023107E1E7F09906A73E0FBAD1645
:100A4100AC151232BC851682851583A3E0B4280843
:100A51009067A57405F080069067A57403F0906710
:100A6100227401F0229067227404F022200F030205
:100A71000B20E540653B604DE54024085438FFE517
:100A81003B54386F60047E0180027E00906A73E0FF
:100A910060047D0180027D00EE5D7003021011850E
:100AA1001682851583E0FEE540131313541F24328B
:100AB100F8A6068F400516E51670020515906A73B3
:100AC100E014F080B39067A5E06406603F30140441
:100AD100D211C214906696E0FCA3E0FDA3E0FEA350
:100AE100E0FFE4FAF9F8EF2401FFEA3EFEE93DFDFB
:100AF100E83CFC90669612246CE4F528D20AD22FC9
:100B0100D2B19067C8E09067C7F080069067C7745C
:100B110041F0C20FC2909067A5E0906722F02230A9
:100B2100B10B300C08906723E09067C7F0C2B13079
:100B31000C0C30B0099067C7E060030210118516F4
:100B410082851583E0FFE540131313541F2432F807
:100B5100A607E54024085438F5400516E51670024D
:100B61000515906A73E014F0D20FD290222006038B
:100B7100020DBFE53F5438653A7003021011E53AA2
:100B810024085438F53A131313541F242AF8E69015
:100B91006949F0200523E0FF1234C78F46906A723D
:100BA100E0D3948050030210119067227407F090F3
:100BB10067C77432F012466A22C291906722E064DC
:100BC100036003020C88906949E0FF1234C78F4625
:100BD100300EA0E546603CC2123023107E1E7F27F6
:100BE1007C697D72906A72E0FB1232BC90669AE079
:100BF100FCA3E0FDA3E0FEA3E0FFE4FAF9F8EF2493
:100C010001FFEA3EFEE93DFDE83CFC90669A1224B4
:100C11006C806490694AE0FF906972E06F60033014
:100C21001342906A72E024FEF0D21230230F7E1E2E
:100C31007F357C697D72E02402FB1232BC906692A2
:100C4100E0FCA3E0FDA3E0FEA3E0FFE4FAF9F8EF86
:100C51002401FFEA3EFEE93DFDE83CFC906692126C
:100C6100246C80133023107E1E7F497C697D729035
:100C71006A72E0FB1232BC9067227407F09067C77A
:100C81007432F012466A22906722E06403702330C6
:100C910023107E1E7F567C697D72906A72E0FB1282
:100CA10032BC9067227407F09067C77432F0124625
:100CB1006A22300344C203906A72E0C3940350195C
:100CC100E014F0E0FB6022D21230231D7E1E7F77FC
:100CD1007C697D721232BC80107E1E7F887C697DAA
:100CE10072906A72E0FB1232BC9067227407F09036
:100CF10067C77432F012466A2290694AE0FF906930
:100D010072E06F60233023107E1E7F497C697D7203
:100D1100906A72E0FB1232BC9067227407F0906710
:100D2100C77432F012466A2290694BE0FF906973F2
:100D3100E06F702E3023107E1E7FB67C697D72902D
:100D41006A72E0FB1232BC301008D212906A72E073
:100D510014F09067227407F09067C77432F012465E
:100D61006A223023107E1E7FC97C697D72906A726F
:100D7100E0FB1232BC201303301016906722740777
:100D8100F09067C77432F0D212906A72E014F0806A
:100D910029906972E090694AF0906973E090694B1B
:100DA100F0906974E090694CF07F021243D490672F
:100DB100227401F09067A57403F012466A22202F75
:100DC1003030230B7E1E7FDAE4FBFDFC1232BCE4E3
:100DD1009067C7F0D206D291906A72F0906B18F0CA
:100DE100906B14F0D204F517D20075136975147263
:100DF100229067C7E0600302101130230A7E1E7F34
:100E0100E9FBFDFC1232BC90669EE0FCA3E0FDA371
:100E1100E0FEA3E0FFE4FAF9F8EF2401FFEA3EFE69
:100E2100E93DFDE83CFC90669E12246C90672274BB
:100E310007F09067C77432F02230100D906722746A
:100E410007F09067C77432F022906B1AE004F0E06B
:100E5100C394204002E4F0906B1AE075F005A424DD
:100E610074F9746A35F0FA7B01906B15EBF0A3EA23
:100E7100F0A3E9F01222D2FF7003020FB0906B15BC
:100E8100E0FBA3E0FAA3E0F9900002740112231839
:100E91009000011222EBFE9000021222EBC39E5041
:100EA10003020F5B906B15E0FBA3E0FAA3E0F9905E
:100EB1000002E412235D90000474011223189000D3
:100EC100031222EBFE9000041222EBD39E401390FA
:100ED1006B15E0FBA3E0FAA3E0F9900004740112A2
:100EE100235D906B15E0FBA3E0FAA3E0F990694A5A
:100EF100EFF09000041222EB441090694BF09067E0
:100F0100A57403F07F021243D4202303020FA97EAC
:100F11001F7F08906B15E0A3E0FAA3E02404F9E435
:100F21003AFCAD017B011232BC7F1E1246547E1F7A
:100F31007F1C906B15E0A3E0FAA3E0AC02FD7B01FE
:100F41001232BC7F1E1246547E1F7F247C697DF2C3
:100F5100906A73E0FB1232BC804E906B15E0FBA3EC
:100F6100E0FAA3E0F91222D290694AF0A37450F09A
:100F71009067A57405F07F021243D430232A7E1FA7
:100F81007F26906B15E0A3E0FAA3E0AC02FD7B01A4
:100F91001232BC7F1E1246547E1F7F247C697DF273
:100FA100906A73E0FB1232BC9067227401F02290C8
:100FB1006B1A74FFF09067227407F09067C7743260
:100FC100F0229067C7E0704830230A7E1F7F3AFB0A
:100FD100FDFC1232BC9067227401F09067A5740584
:100FE100F0851115851216906A73E510F022301202
:100FF100169067C7E070197E1F7F4DFBFDFC123212
:10100100BCE4906722F022E49067C7F0906722F079
:0110110022BC
:0B465F00301105C2117F01227F0022F4
:03467100C2AE22B4
:103CDF00021012E493A3F8E493A34003F68001F2D9
:103CEF0008DFF48029E493A3F85407240CC8C333E6
:103CFF00C4540F4420C8834004F456800146F6DFB5
:103D0F00E4800B0102040810204080903A21E47EE9
:103D1F00019360BCA3FF543F30E509541FFEE493A9
:103D2F00A360010ECF54C025E060A840B8E493A370
:103D3F00FAE493A3F8E493A3C8C582C8CAC583CA9B
:103D4F00F0A3C8C582C8CAC583CADFE9DEE780BE53
:013AE00000E5
:1022D200BB010689828A83E0225002E722BBFE020A
:0922E200E32289828A83E493223D
:1022EB00BB010CE58229F582E5833AF583E02250A8
:1022FB0006E92582F8E622BBFE06E92582F8E222F2
:0D230B00E58229F582E5833AF583E493220B
:10231800BB010FF8E58229F582E5833AF583E028C9
:10232800F0225009C58229F8E58226F622BBFE096B
:10233800C58229F8E22582F222F8EA2583F583E9A5
:03234800932822B5
:10234B00BB010689828A83F0225002F722BBFE0171
:02235B00F3226B
:10235D00F8BB010DE58229F582E5833AF583E8F0B6
:10236D00225006E92582C8F622BBFE05E92582C862
:02237D00F2224A
:10237F0075F008758200EF2FFFEE33FECD33CDCC15
:10238F0033CCC58233C5829BED9AEC99E582984098
:10239F000CF582EE9BFEED9AFDEC99FC0FD5F0D675
:1023AF00E4CEFBE4CDFAE4CCF9A88222B800C1B99F
:1023BF000059BA002DEC8BF084CFCECDFCE5F0CBDD
:1023CF00F97818EF2FFFEE33FEED33FDEC33FCEB16
:1023DF0033FB10D703994004EB99FB0FD8E5E4F9D1
:1023EF00FA227818EF2FFFEE33FEED33FDEC33FCBE
:1023FF00C933C910D7059BE99A4007EC9BFCE99AB2
:10240F00F90FD8E0E4C9FAE4CCFB2275F010EF2FF6
:10241F00FFEE33FEED33FDCC33CCC833C810D707F6
:10242F009BEC9AE899400AED9BFDEC9AFCE899F831
:0E243F000FD5F0DAE4CDFBE4CCFAE4C8F922C4
:0E244D00C3E49FFFE49EFEE49DFDE49CFC22A0
:10245B00EB9FF5F0EA9E42F0E99D42F0E89C45F0D7
:01246B00224E
:0C246C00ECF0A3EDF0A3EEF0A3EFF022E3
:10247800A8828583F0D083D08212248F12248F12F1
:10248800248F12248FE473E493A3C583C5F0C58316
:10249800C8C582C8F0A3C583C5F0C583C8C582C8AE
:0124A8002211
:101F7600E55A244EF8E6055A22784B302D02784E63
:101F8600E475F0011224F80222D22026EB7F2ED22D
:101F9600268018EF540F2490D43440D4FF302A0BF7
:101FA600EF24BFB41A0050032461FFE55B600215FD
:101FB6005B055EE55E7002055D302D0D784BE475C0
:101FC600F0011224F8EF02234B0244207403D22DB1
:101FD6008003E4C22DF55A8B4B8A4C894DE4F55BA0
:101FE600F55DF55EE55B60077F20121FB180F57534
:101FF6005CFFC227C226C228C229C22BC22CC22E0F
:10200600121F7FFF700D302D057F00121FC2AF5EBD
:10201600AE5D22B4255FC2D5C22A121F7FFF24D02F
:10202600B40A00501A75F00A785B30D50508B6FF79
:102036000106C6A426F620D5047002D22980D9242A
:10204600CFB41A00EF5004C2E5D22A0221C2D22729
:1020560080C6D22680C0D22880BCD2D580BAD22BE8
:1020660080B47F20121FB12028077401B55B0040A1
:10207600F1121F76FF121FB1021FEAD22ED22C8058
:1020860095121F76FB121F76FA121F76F94A4B70CD
:102096000679937A227BFF20282EE55B602A7E0054
:1020A6008E827583001222EB60060EEE655C70F080
:1020B600C2D5EBC0E0EAC0E0E9C0E0EE122209D0EA
:1020C600E0F9D0E0FAD0E0FB1222D2FF60AAEBC022
:1020D600E0EAC0E0E9C0E0121FB1D0E02401F9D087
:1020E600E03400FAD0E0FBE55C0460DCD55CD98026
:1020F600877BFF7A227905D228809C791080027925
:1021060008C22CC22E8008D2D5790A8004790AC268
:10211600D5E55C047002F55CE4FAFDFEFF121F765D
:10212600FC7B08202713121F76FD7B1030260A122F
:102136001F76FE121F76FF7B20EC3382D592D55098
:1021460013C3E43026069FFFE49EFEE42027039D8A
:10215600FDE49CFCE4CBF8C227EC700CCFCECDCCD2
:10216600E824F8F870F38017C3EF33FFEE33FEED83
:1021760033FDEC33FCEB33FB994002FB0FD8E9EB64
:10218600302705F8D0E0C448B227C0E00AEC4D4E2F
:102196004F78207B0070C2EAB55C0040BCC0E012FC
:1021A600220BD0F0D0E0202704C4C0E0C4B227C080
:1021B600F0121F9AD0F0D5F0EB021FEA1225572035
:1021C600875321015820584C20544221054F210D98
:0F21D60044210D49206D4321135520F74620F772
:1021E5004520F74722B350205C2D20602E20832BFD
:1021F500206423208120229C2A201C480000207B6B
:102205003F3F3F00790AA2D5202914302B09B91088
:10221500020404B9080104A2D5202C0250010420AF
:1022250028689228B55B005034C0E07F203029191A
:102235007F30A228722C722B500F122262C228C244
:102245002CC22BC22E7F30800F302B03E9C0E01249
:102255001FB1302B03D0E0F9D0E0B55BCC302B17A4
:102265007F30B9100C121FB17F58302A077F788054
:1022750003B90803121FB13028057F2D021FB17F56
:1022850020202EF87F2B202CF322922880CF286E39
:10229500756C6C2900D227121F763027F8C2277873
:1022A5005B30D50108F602201C2D50434958121FFA
:1022B500762403B405004001E49022AE93121FA2D8
:0D22C500743A121FA2D229755B0402210198
:102B5E008B488A49894AE4F554F553F552F551F5F7
:102B6E004FF550E54C454D454B6012EBC0E0EAC0C9
:102B7E00E0E9C0E0AB4BAA4CA94D122508AB4805C5
:102B8E004AE54AAA497002054914F91222D2F555AE
:102B9E00C394094007E555D3940D40E1E5556420F3
:102BAE0060DBE555B42D054350038016E555B42B77
:102BBE0005435001800C74FF254AF54A74FF3549D0
:102BCE00F549E54E60046410703FAB48AA49A94A26
:102BDE001222D264306009E54E702E754E0A80299D
:102BEE009000011222EBFF64786004EFB458134397
:102BFE005001754E107402254AF54AE43549F549DF
:102C0E008007E54E7003754E08AB48054AE54AAAA3
:102C1E00497002054914F91222D2F555C394614048
:102C2E000AE555D3947A50035355DF74D02555F5E4
:102C3E0055C3940A400CE5559411406D74F9255511
:102C4E00F555E555D3954E50604350018554598541
:102C5E005358855257855156AF4E7E00E4FCFDAB5E
:102C6E0054AA53A952A8511224A9C8ECC8C9EDC937
:102C7E00CAEECACBEFCBE4FCFDFEEB2555F554EEC8
:102C8E003AF553ED39F552EC38F551AF54AE53AD2C
:102C9E0052FCAB59AA58A957A856D312245B50031D
:102CAE00022C17435004022C17E55020E003E48059
:102CBE002DE54C454D454B601EAB48E54A24FFF9CA
:102CCE00E54934FFFAEBC0E0EAC0E0E9C0E0AB4B07
:102CDE00AA4CA94D122508E55030E20774FFFFFEFD
:102CEE00FDFC22E550AF54AE53AD52AC5130E10372
:042CFE0002244D223D
:1024A900E88FF0A4CC8BF0A42CFCE98EF0A42CFCD2
:1024B9008AF0EDA42CFCEA8EF0A4CDA8F08BF0A450
:1024C9002DCC3825F0FDE98FF0A42CCD35F0FCEBAF
:1024D9008EF0A4FEA9F0EB8FF0A4CFC5F02ECD3974
:0F24E900FEE43CFCEAA42DCE35F0FDE43CFC22E1
:1024F800FAE6FB0808E6F925F0F618E6CA3AF622E5
:10250800BB011A89828A83D0F0D0E0F8D0E0F9D0F4
:10251800E0FAD0E0FBE8C0E0C0F00225865016E9FA
:10252800F8D083D082D0E0F9D0E0FAD0E0FBC082C6
:10253800C08302257DBBFE16E9F8D083D082D0E0A7
:0F254800F9D0E0FAD0E0FBC082C08302258F22D9
:10255700D083D082F8E4937012740193700DA3A313
:1025670093F8740193F5828883E473740293686027
:06257700EFA3A3A380DF27
:09257D00EBF608EAF608E9F62283
:09258600EBF0A3EAF0A3E9F02256
:09258F00EBF208EAF208E9F2227D
:00000001FF
